:020000040000FA
:0400000069303A2801
:08000800A000030EA100831209
:1000100005191028831601178312B23081002B288E
:1000200083160113831203140B190310A80DA90DD5
:10003000AA0DAB0DAC0DAC16FF302C02031D2B2806
:10004000FA302B02031D2B2831152A08AF0029088E
:10005000AE002808AD008B100B11210E8300A00EFE
:04006000200E090065
:0C007400203084008001840A6030040207
:10008000031C3C281230B0003E228316FF23900050
:10009000831283160C308505870183128501870141
:1000A000073099000030831691008312C830831600
:1000B0008100831231309000003083168C0083124F
:1000C00010308B00831600309B001C141A0883121A
:1000D000BC00851DBE233C1C7528831610309B0078
:1000E0001C141A088312BD001F23831620309B00A6
:1000F0001C141A088312C1000130C1080319C10081
:1001000081018E018F010B118B100B108C018B174D
:10011000982031199B202222B30B962803108519B1
:100120000314B90DF03039020319A32130238828B4
:1001300064003210080031110130B7008514400806
:10014000013ECE000F08CF008B13203037078316F7
:100150009B001C141A088312A40010303707831662
:100160009B001C141A088312A300A6000230A606E6
:100170000030370783169B001C141A088312A20054
:10018000A7000130A7068B17321CCC28220903399F
:10019000A200A309A409A50924082F02031D9D2973
:1001A00023082E02031D362922082D02031D9D2936
:1001B00001303702031DE3283C19E2283D18E328EB
:1001C0003D143E143F2202303702031DEE283C1935
:1001D000ED28BD18EE28BD143E144C220330370222
:1001E000031DF9283C19F8283D19F9283D153E143E
:1001F000592204303702031D04293C190329BD1973
:100200000429BD153E14662205303702031D0F294F
:100210003C190E293D1A0F293D163E147322063053
:100220003702031D1A293C191929BD1A1A29BD16AE
:100230003E14802207303702031D25293C1924294A
:100240003D1B25293D173E148D2208303702031D22
:1002500030293C192F29BD1B3029BD173E149A2285
:1002600009303702031D36293E14A72226082E0224
:10027000031D9D2927082D02031D9D2901303702EA
:10028000031D49293C1948293D1C49293D103E14AC
:10029000CE2202303702031D54293C195329BD1CBC
:1002A0005429BD103E14D22203303702031D5F29AA
:1002B0003C195E293D1D5F293D113E14D6220430B4
:1002C0003702031D6A293C196929BD1D6A29BD1120
:1002D0003E14DA2205303702031D75293C197429B2
:1002E0003D1E75293D123E14DE2206303702031DE5
:1002F00080293C197F29BD1E8029BD123E14E222AF
:1003000007303702031D8B293C198A293D1F8B2991
:100310003D133E14E62208303702031D96293C198E
:100320009529BD1F9629BD133E14EA2209303702D4
:10033000031D9C293E14EE229D29B70A0A3037027C
:1003400003180800A4280130B600B300B400B500BB
:10035000B70085018701B1139820B30BE929031079
:1003600085190314B90DF03039020319102AB41F8E
:100370008510B40BE929013037020319F22202304B
:1003800037020319F622033037020319FA22043028
:1003900037020319FE220530370203190223063003
:1003A0003702031906230730370203190A230830DE
:1003B000370203190E2309303702031912233708B5
:1003C000B6080319B6000319E7298514B603963059
:1003D000B400311DAC293111321CF3292D09033928
:1003E000AD00AE09AF092F1CAC298E018F010C1C8A
:1003F000AC290C102E1EAC298B1320303707BB0004
:100400002F08BA002B2210303707BB002E08BA0085
:100410002B2200303707BB002D08BA002B228B1788
:1004200085018701083037022030031985002A3002
:1004300003198700B70AB6010A303702031CAC293A
:100440001F2308003E1C08003E101030BB003D0872
:10045000BA002B2208008B133A0883161C159A0049
:100460003B089B0055309D00AA309D009C14640001
:100470009C18372A1C1183128B17080008003C199E
:10048000871640083C1D40034107D0000F08D100EB
:10049000BC1919233D1408003C19071640083C1DDF
:1004A00040034107D2000F08D300BC191923BD1423
:1004B00008003C19871540083C1D40034107D40043
:1004C0000F08D500BC1919233D1508003C19051665
:1004D00040083C1D40034107D6000F08D700BC1957
:1004E0001923BD1508003C19851640083C1D400322
:1004F0004107D8000F08D900BC1919233D16080080
:100500003C19071540083C1D40034107DA000F085D
:10051000DB00BC191923BD1608003C1987144008DC
:100520003C1D40034107DC000F08DD00BC19192306
:100530003D1708003C19071440083C1D40034107C3
:10054000DE000F08DF00BC191923BD170800BC1915
:1005500008003C1DAF2A303085043F3087048E01EF
:100560008F01C001D001D201D401D6010130D800E1
:10057000DA00DC00DE004030D1008030D300C03033
:10058000D500FF30D7004030D9008030DB00C030CC
:10059000DD00FF30DF00FF30BD00080087128E0154
:1005A0008F01080007128E018F01080087118E014C
:1005B0008F01080005128E018F01080085128E013F
:1005C0008F01080007118E018F01080087108E012E
:1005D0008F01080007108E018F01080019238E017A
:1005E0008F0108000708203A870008000708103A22
:1005F000870008000708083A870008000508103A35
:10060000850008000508203A850008000708043A1C
:10061000870008000708023A870008000708013A27
:10062000870008000508303A850007083F3A870030
:100630000800CF308505C0308705BD0108003D1892
:100640008716BD1807163D198715BD1905163D1AE1
:100650008516BD1A07153D1B8714BD1B071408001E
:100660003C19342B3D1C402B50084002031D402BED
:1006700051080F02031C402B3C1987123C1D8716A2
:100680003C19442BBD1C502B52084002031D502B1B
:1006900053080F02031C502B3C1907123C1D071670
:1006A0003C19542B3D1D602B54084002031D602B48
:1006B00055080F02031C602B3C1987113C1D871540
:1006C0003C19642BBD1D702B56084002031D702B76
:1006D00057080F02031C702B3C1905123C1D051610
:1006E0003C19742B3D1E802B58084002031D802BA3
:1006F00059080F02031C802B3C1985123C1D8516DE
:100700003C19842BBD1E902B5A084002031D902BD0
:100710005B080F02031C902B3C1907113C1D0715A9
:100720003C19942B3D1FA02B5C084002031DA02BFD
:100730005D080F02031CA02B3C1987103C1D871479
:100740003C19A42BBD1FB02B5E084002031DB02B2B
:100750005F080F02031CB02B3C1907103C1D071447
:100760004E084002031DB92B4F080F02031CB92B82
:1007700085100C1C08000C10C00A0800B601B3015B
:10078000B4013C1CC62BBC01BC14D22BBC1CCB2B13
:10079000BC013C15D22B3C1DD02BBC01BC15D22B6F
:1007A000BC013C143C08B6006400D62BD72BD82BD8
:1007B000D92BDA2BB41B8716B41F8712B30BD42B9B
:1007C000B40BD42B0310B60CB608031DD42B003089
:0A07D000BB003C08BA002B22080011
:084000000800030003000200A8
:02400E00CC01E3
:10420000010078007A007C007E007B0079007F004E
:104210007D007A0078007E007C00FF00FF00FF0038
:104220000000F200F600FA00FE00F200F600FA00CC
:10423000FE00F200F600FA00FE00FF00FF00FF00A3
:10424000010005000500050005000900090009003E
:1042500009000D000D000D000D00FF00FF00FF0024
:10426000FF00FF00FF00FF00FF00FF00FF00FF0056
:10427000FF00FF00FF00FF00FF00FF00FF00FF0046
:10428000FF00FF00FF00FF00FF00FF00FF00FF0036
:10429000FF00FF00FF00FF00FF00FF00FF00FF0026
:1042A000FF00FF00FF00FF00FF00FF00FF00FF0016
:1042B000FF00FF00FF00FF00FF00FF00FF00FF0006
:1042C000FF00FF00FF00FF00FF00FF00FF00FF00F6
:1042D000FF00FF00FF00FF00FF00FF00FF00FF00E6
:1042E000FF00FF00FF00FF00FF00FF00FF00FF00D6
:1042F000FF00FF00FF00FF00FF00FF00FF00DD00E8
:00000001FF
